:0400000030EF3FF0AE
:107E600000016AEF3FF0016E9EA8FED701C0ADFF92
:107E70001200AC98AC9CAB8E810EAF6EAC84B89601
:107E8000948E948CAB88AC8A120001500210D8B446
:107E9000120003C004F00F0E041601C0D9FF02C087
:107EA000DAFFDF500418F00B0418DF6E12000150E7
:107EB0000210D8B4120003C005F00F0E051601C061
:107EC000D9FF02C0DAFF053ADF5005180F0B05187D
:107ED000DF6E12000E0E066E000E076E000E096EAB
:107EE000000E086E3C0E0A6E7F0E0B6E81EC3FF0AA
:107EF00039EC3FF00E0E026E000E036EBCEC3FF04C
:107F0000F9D706500710D8B41200030E06240C6EE1
:107F1000000E07200D6E0C500D10D8B4120006C0D4
:107F200001F007C002F0080E036E45EC3FF006C0FA
:107F300001F007C002F008C003F009C004F057ECDC
:107F40003FF020EE03F00650D9260750DA220AC08F
:107F5000DFFF20EE04F00650D9260750DA220BC0CE
:107F6000DFFF20EE01F00650D9260750DA22020E7C
:107F7000DE6E000EDD6E120002500310D8B4120047
:107F8000030E0224046E000E0320056E045005103B
:107F9000D8B4120020EE01F00250D9260350DA22A4
:107FA000DECF06F0DDCF07F0030E0224086E000ED0
:107FB0000320096E02C0D9FF03C0DAFFDF380F0BC0
:107FC000046E02C0D9FF03C0DAFFDF500F0B056E4D
:107FD0000538F00B041033EC3FF009D008C0D9FF8E
:107FE00009C0DAFFDF5033EC3FF0084A092A0606E1
:107FF000D8A007060628F2E10728D8B41200EED769
:020000040020DA
:08000000FFFFFFFFFFFFFFFF00
:020000040030CA
:0E000000FF251F3FFFBF85FF0FC00FE00F4021
:00000001FF
